:020000040000FA
:060000007AEF08F0120087
:060800007AEF08F012007F
:06082A000100281100008E
:08083000000200003A00000084
:08083800D9CFE6FFE1CFD9FFA3
:10084000040EE126DE6ADE6ADE6ADD6ADD52DD5212
:10085000FD0EDBCF00F0FE0EDBCF01F0026A036A73
:1008600001AE02D002680368D9CFE9FFDACFEAFF10
:10087000030EEB500318E8AE02D0033408D000504A
:10088000EE5C0150EE580250EE580350EE580FE265
:100890000C0EE66E5AEC08F0E552D9CFE9FFDACF3C
:1008A000EAFFEE2A000EEE22EE22EE22D1D7040E4F
:1008B000E15C02E2E16AE552E16EE552E7CFD9FF81
:1008C00012000F0EC16E070EB46E936A300E926E58
:1008D0000F0E946EF19E1200D9CFE6FFE1CFD9FF43
:1008E000020EE1268250020B01E0010E080DF3CF4B
:1008F00002F08250010B040DF3CF01F08050200B69
:1009000001E0010EE824006E8050100B01E0010EA2
:10091000002401240224DE6EDD6ADECF00F0DDCF8C
:1009200001F000C0F3FF01C0F4FF020EE15C03E23E
:1009300000D0E16AE552E16EE552E7CFD9FF12003F
:100940008092320EE66E88EC08F0E5528084320E1A
:10095000E66E88EC08F0E5528094320EE66E88EC84
:1009600008F0E55212008082010EE66EE66A64DF4E
:10097000E552E5528084010EE66EE66A5DDFE552DF
:10098000E5528094010EE66EE66A56DFE552E552C6
:100990001200380E816ED4DF320EE66EE66A4CDF4E
:1009A000E552E552010E816ECBDF320EE66EE66A4D
:1009B00043DFE552E5520D0E816EC2DF320EE66E68
:1009C000E66A3ADFE552E552060E816EB9DF320E75
:1009D000E66EE66A31DFE552E5521200010E816EE5
:1009E000AFDF0A0EE66EE66A27DFE552E552120037
:1009F000D9CFE6FFE1CFD9FF020E816EA1DF0A0E4B
:100A0000E66EE66A19DFE552E552FD0EDBCFE6FF42
:100A1000FE0EDB50280DF350E552E724E76EFE0E84
:100A2000E7CFDBFFFD0EDB6AFE0EDB50F36EFD0E43
:100A3000DBCFF4FFF350F45C0BE2140E816E80DF29
:100A4000320EE66E88EC08F0E552FD0EDB2AECD79C
:100A5000E552E7CFD9FF1200D9CFE6FFE1CFD9FFAA
:100A6000FE0EDB50816E7FDF010EE66EE66AE4DE8D
:100A7000E552E552E552E7CFD9FF1200D9CFE6FFA4
:100A8000E1CFD9FFFD0EDBCFE9FFFE0EDBCFEAFFA2
:100A9000EF500EE0FD0EDBCFE9FFDB2AFE0EDBCFD1
:100AA000EAFF01E3DB2AEF50E66ED6DFE552EAD734
:100AB000E552E7CFD9FF12000001646B300E926E51
:100AC000F00E936EEF0E606F60C081FF040E616FD9
:100AD0006151000821E26051FE0BE842606F60C086
:100AE00081FF050EE66EE66AA7DEE552E55281500B
:100AF000100B09E08150200B06E08150400B03E011
:100B00008150800B01E10AD80001640502E16551C2
:100B100004D06105616FDCD7CFD71200F00E936E61
:100B200081CF63F000016315626F0F0E6015606F77
:100B300060516211606F81CF63F0F00E6315626FD8
:100B4000F00E625D01E0F7D7936A06D866C065F0E3
:100B50000001010E646F12000001676B100E675DEB
:100B600014E26751EA6A000FE96E020EEA22EF50C2
:100B7000605D08E16751EA6A100FE96E020EEA2231
:100B8000EFCF66F06729676FE9D766C081FF640E13
:100B9000E66EE66A51DEE552E55212000001686B2E
:100BA000070E685D1DE288DF0001696F6851EA6A1F
:100BB0006A0FE96E000EEA2269C0EFFF6851EA6A27
:100BC0006A0FE96E000EEA22EF50460802E108D0F3
:100BD00004D069C0E6FF40DFE5520001682BE0D792
:100BE0006851EA6A6A0FE96E000EEA22EF6A1200A3
:100BF0000001686B070E685D16E26851EA6A6A0FC9
:100C0000E96E000EEA22EF50E66E26DFE5520001A3
:100C10006829EA6A6A0FE96E000EEA22EF5001E1E4
:100C200002D0682BE7D71200D9CFE6FFE1CFD9FF7A
:100C3000E652F250800B01E0010EDF6EF29EA69E9E
:100C4000A69CA684FE0EDB50A96EFD0EDB50A86E9E
:100C5000550EA76EAA0EA76EA682A6B2FED7A694C0
:100C6000DF50E8B0F28EE8A0F29EE552E552E7CF01
:100C7000D9FF1200D9CFE6FFE1CFD9FFA69CA69EEF
:100C8000FE0EDB50A96EA680A85000D0E552E7CF3B
:100C9000D9FF12004D0EE66EE66A6C0EE66EA3EC0E
:100CA00007F0E552E552E5521200D9CFE6FFE1CF59
:100CB000D9FF040EE126DE6ADE6ADE6ADD6ADD52F5
:100CC000DD52D9CFE9FFDACFEAFFD890030EEB501F
:100CD000000A08E6400EEE5C0D0EEE58030EEE58CC
:100CE000000EEE5811E29EAA04D024EC08F00ED0BB
:100CF00001D000D0D9CFE9FFDACFEAFFEE2A000E0B
:100D0000EE22EE22EE22DDD7000E00D0006E040EA1
:100D1000E15C02E2E16AE552E16E0050E552E7CFA4
:100D2000D9FF1200D9CFE6FFE1CFD9FFE6529EAA44
:100D3000FED724EC08F0DF6EDFCFE6FF43EC08F0CF
:100D4000E552F5D7DF5000D0E552E552E7CFD9FFA5
:100D50001200D9CFE6FFE1CFD9FFE6529EAAFED717
:100D600024EC08F0DF6EDF5000D0E552E552E7CF0B
:100D7000D9FF1200A6DD0DDE31DE200EE66E020E7A
:100D8000E66E7CDEE552E5520001876B886B080E4B
:100D900088AF02D0D89003D0875D000E885917E243
:100DA00087C0E9FF88C0EAFFD890E936EA362A0E04
:100DB000E926020EEA22EECFE6FFEFCFE6FF09D8E2
:100DC000E552E5520001872B000E8823E0D7D4D7E7
:100DD0001200D9CFE6FFE1CFD9FF020EE126FEDDFA
:100DE0002A0EE66E39DEE552DE6ADD6ADECF00F0FD
:100DF000DDCF01F0D890015004E6080E005C000E33
:100E0000015816E2FD0EDBCF00F0FE0EDBCF01F045
:100E1000DE500024F66EDD500120F76E0800F5501C
:100E2000E66E1ADEE552DF2A010E01E3DB2ADED789
:100E3000E66A010EE66EDCDDE552E552070EDE6E77
:100E4000DD6ADECF00F0DDCF01F0D890015004E67E
:100E50000E0E005C000E015816E2FD0EDBCF00F016
:100E6000FE0EDBCF01F0DE500024F66EDD500120D7
:100E7000F76E0800F550E66EEFDDE552DF2A010E51
:100E800001E3DB2ADED7E80EE66E030EE66ED4DC65
:100E9000E552E552020EE15C02E2E16AE552E16EE2
:080EA000E552E7CFD9FF120073
:080EA8002A0EF66E080EF76E2B
:100EB000000EF86E00010900F550906F0900F55022
:100EC000916F03E1906701D03DD00900F5508B6F21
:100ED0000900F5508C6F0900F5508D6F090009006D
:100EE000F550E96E0900F550EA6E090009000900A5
:100EF000F5508E6F0900F5508F6F09000900F6CF8D
:100F000092F0F7CF93F0F8CF94F08BC0F6FF8CC03F
:100F1000F7FF8DC0F8FF00018E5302E18F5307E009
:100F20000900F550EE6E8E07F8E28F07F9D792C0F0
:100F3000F6FF93C0F7FF94C0F8FF00019007000E82
:060F4000915BBFD7120017
:0A0F4600D9CFE6FFDACFE6FFE1CFD6
:100F5000D9FFE2CFDAFFAC6AAB6AFD0EDBB0AC883A
:100F6000DBA202D0AC8CAB8CDBB4AC8EDBA602D0A7
:100F7000AB8801D0AB8ADBB8AC849E98DBBAAB8679
:100F8000DBAC02D09D8A01D09D9A9E9ADBAE02D046
:100F90009D8801D09D98FB0EDB50AF6EFB0EFC0EC2
:100FA000DBCF01F001C000F0016A0050B06EAC8AE6
:100FB000AB8E949C948EAC50100B04E0AC50800B24
:100FC00001E1948CE552E5CFDAFFE7CFD9FF1200BB
:100FD0004A4F5345204845524E414E44455A0050D1
:100FE00041424C4F204A494D454E455A2000504100
:100FF0004F4C4120455350494E4F5A41004A4149B8
:101000004D4520424554414E5A4F53004C5549538B
:1010100020524F424C45444F202000524F424552EF
:10102000544F204C494D4F4E20004A4F484E2043CC
:10103000415354454C41522000444149535920509A
:081040004552455A2020200012
:08104800D9CFE6FFDACFE6FF85
:10105000E1CFD9FFE2CFDAFFE652F20E02013A17F2
:10106000ABAC03D03A91ABB03A81ABB43A85ABB2FA
:101070003A87AE50DF6EDF50E552E552E5CFDAFF3A
:06108000E7CFD9FF1200CA
:0A108600D9CFE6FFDACFE6FFE1CF95
:10109000D9FFE2CFDAFFACAC04D0AC9002013AB396
:1010A000AC80FD0EDB50AD6EE552E5CFDAFFE7CF49
:0410B000D9FF120052
:0C10B400FF0EE350066E480E01D04C0EFB
:1010C000E76EE72EFED7E76AE72EFED7062EF7D7A4
:0410D000000012000A
:0C10D400000EF36E00EE00F0080E01D8D4
:1010E0001200EA6002D0EE6AFCD7F350E960120009
:0410F000EE6AFCD7D1
:0C10F40012EE40F022EE40F0F86A059C7D
:1011000054EC07F093EC08F0BAEC06F0FBD71200B1
:10111000FF0EE350E84E1200000000D000D000D0D7
:06112000E82EFAD71200D0
:021126001200B5
:08112800EEEDEBE7DEDDDBD7A5
:10113000BEBDBBB77E7D7B77303132333435363739
:1011400038394142434445464C495354413A2020A2
:101150002000D00FDF0FEE0FFD0F0C101B102A1018
:02116000391044
:00000001FF
